:100000000C9474000C949C000C949C000C949C0028
:100010000C949C000C949C000C949C000C949C00F0
:100020000C949C000C949C000C949C000C949C00E0
:100030000C949C000C949C000C949C000C949C00D0
:100040000C94E7020C949C000C9457030C9431031D
:100050000C949C000C949C000C949C000C949C00B0
:100060000C949C000C949C000000000024002700CD
:100070002A0000000000250028002B0004040404CE
:100080000404040402020202020203030303030342
:10009000010204081020408001020408102001021F
:1000A00004081020746869732069732061207465E6
:1000B0007374206F66206D616B696E672073757253
:1000C000652064617461206D616B657320697420C3
:1000D000696E746F20746865207465787420736528
:1000E000676D656E7400F60311241FBECFEFD8E074
:1000F000DEBFCDBF11E0A0E0B1E0E8EBFAE002C066
:1001000005900D92A231B107D9F721E0A2E1B1E04B
:1001100001C01D92A83BB207E1F710E0C4E7D0E0B0
:1001200004C02197FE010E942304C337D107C9F7F9
:100130000E9489030C942E040C940000FFFFFFFF23
:10014000FFFFFFFFFFFFFFFFFFFFFFFFFFFFFFFFBF
:10015000FFFFFFFFFFFFFFFFFFFFFFFFFFFFFFFFAF
:10016000FFFFFFFFFFFFFFFFFFFFFFFFFFFFFFFF9F
:10017000FFFFFFFFFFFFFFFFFFFFFFFFFFFFFFFF8F
:10039000FFFFFFFFFC01538D448D252F30E0842F9C
:1003A00090E0821B930B541710F0CF96089501979D
:1003B0000895FC01918D828D981761F0828DDF0187
:1003C000A80FB11D5D968C91928D9F5F9F73928F48
:1003D00090E008958FEF9FEF0895FC01918D828D3D
:1003E000981731F0828DE80FF11D858D90E008950A
:1003F0008FEF9FEF0895FC01918D228D892F90E062
:10040000805C9F4F821B91098F7399270895FC018F
:10041000848DDF01A80FB11DA35ABF4F2C91848D8D
:1004200090E001968F739927848FA689B7892C93C2
:10043000A089B1898C9180648C93938D848D98135D
:1004400006C00288F389E02D80818F7D8083089526
:10045000EF92FF920F931F93CF93DF93EC0181E014
:10046000888F9B8D8C8D981305C0E889F9898081D0
:1004700085FD24C0F62E0B8D10E00F5F1F4F0F730C
:100480001127E02E8C8DE8120CC00FB607FCFACFB6
:10049000E889F989808185FFF5CFCE010E940702A6
:1004A000F1CF8B8DFE01E80FF11DE35AFF4FF08273
:1004B0000B8FEA89FB898081806207C0EE89FF8902
:1004C0006083E889F98980818064808381E090E09D
:1004D000DF91CF911F910F91FF90EF900895CF93EF
:1004E000DF93EC01888D8823C9F0EA89FB8980813C
:1004F00085FD05C0A889B9898C9186FD0FC00FB60E
:1005000007FCF5CF808185FFF2CFA889B9898C914E
:1005100085FFEDCFCE010E940702E7CFDF91CF919B
:1005200008958BE191E00E94FB0121E0892B09F401
:1005300020E0822F089580E090E0892B29F00E942E
:10054000910281110C9400000895CF92DF92EF92F6
:10055000FF920F931F93CF93DF936C017A018B016E
:10056000C0E0D0E0CE15DF0581F0D8016D918D019E
:10057000D601ED91FC910190F081E02DC601099525
:10058000892B11F02196EECF7E01C701DF91CF912B
:100590001F910F91FF90EF90DF90CF9008950895F5
:1005A00080E090E00895009769F0FC010190002040
:1005B000E9F73197AF01481B590BBC018BE191E082
:1005C0000C94A50280E090E008950E9429041F92F7
:1005D0000F920FB60F9211242F933F938F939F93F7
:1005E000AF93BF938091170190911801A0911901C9
:1005F000B0911A013091160123E0230F2D3720F41A
:100600000196A11DB11D05C026E8230F0296A11D6C
:10061000B11D209316018093170190931801A093A8
:100620001901B0931A018091120190911301A091C8
:100630001401B09115010196A11DB11D8093120105
:1006400090931301A0931401B0931501BF91AF9142
:100650009F918F913F912F910F900FBE0F901F9000
:1006600018951F920F920FB60F9211242F933F935C
:100670004F935F936F937F938F939F93AF93BF93AA
:10068000EF93FF938BE191E00E940702FF91EF91BE
:10069000BF91AF919F918F917F916F915F914F919A
:1006A0003F912F910F900FBE0F901F9018951F92A2
:1006B0000F920FB60F9211242F938F939F93EF9366
:1006C000FF93E0912B01F0912C018081E0913101A9
:1006D000F091320182FD12C09081809134018F5FD0
:1006E0008F7320913501821751F0E0913401F0E0D1
:1006F000E55EFE4F958F8093340101C08081FF91AC
:10070000EF919F918F912F910F900FBE0F901F909F
:100710001895789484B5826084BD84B5816084BD69
:1007200085B5826085BD85B5816085BD80916E008F
:10073000816080936E0010928100809181008260C0
:1007400080938100809181008160809381008091FD
:1007500080008160809380008091B10084608093EC
:10076000B1008091B00081608093B00080917A00E8
:10077000846080937A0080917A00826080937A000E
:1007800080917A00816080937A0080917A008068FD
:1007900080937A001092C100EDE9F0E02491E9E83D
:1007A000F0E08491882399F090E0880F991FFC0174
:1007B000E859FF4FA591B491FC01EE58FF4F859188
:1007C00094918FB7F894EC91E22BEC938FBF84EA6D
:1007D00090E00E94D3028CE391E00E94D3028CE56A
:1007E00098E00E94D3020E949B02FDCFEBE1F1E072
:1007F0001382128288EE93E0A0E0B0E084839583B8
:10080000A683B78384E091E09183808385EC90E0B8
:100810009587848784EC90E09787868780EC90E0CA
:10082000918B808B81EC90E0938B828B82EC90E0BB
:10083000958B848B86EC90E0978B868B118E128E35
:10084000138E148E0895EE0FFF1F0590F491E02D86
:10085000099481E090E0F8940C942E04FFFFFFFFD0
:10086000FFFFFFFFFFFFFFFFFFFFFFFFFFFFFFFF98
:10087000FFFFFFFFFFFFFFFFFFFFFFFFFFFFFFFF88
:10088000FFFFFFFFFFFFFFFFFFFFFFFFFFFFFFFF78
:10089000FFFFFFFFFFFFFFFFFFFFFFFFFFFFFFFF68
:020AC800ED013E
:00000001FF
